:100000000C942A001895000018950000189500001F
:10001000189500001895000018950000189500002C
:10002000189500001895000018950000189500001C
:10003000189500000C947D25189500001895000077
:1000400018950000189500001895000018950000FC
:10005000189500008FE58DBFC0E2E4E94E2E88E0E0
:100060008EBFD8E0F7E05F2EEEEFF7E0A0E6B0E05D
:10007000A89584B7082E877F84BF88E1992781BD22
:1000800091BD88278D933197E9F783E389B980E0A3
:1000900080BD88E18AB96624579A7894D29ADA9812
:1000A0008C988D9A95988E9A96988F988A9A92980D
:1000B00080917A02806480937A02E0E0F0E0ADED16
:1000C000B2E09CE00E946C26A19AA998A69AAE9AEA
:1000D000D59AD69AD79AAAEEB2E0E0E4FDE40E945F
:1000E0009A240E94612482E2A9EFB2E08D938827CE
:1000F0008C930E94B4080E94BF080E941D090E94B0
:100100001D095A924A9280E0A42DB52D8C9381E06E
:100110000E94F7235A924A9280E0A42DB52D8C9329
:1001200081E00E94F7230E94B009249682E00E9499
:10013000F3235A924A92A42DB52DEEE4FDE40E94D9
:100140009A248CE00E94F7230E94610A22968CE098
:100150000E94F32384E690E00E9485245A924A92FA
:1001600080E0A42DB52D8C9381E00E94F7235A9254
:100170004A9281E0A42DB52D8C9381E00E94F72353
:100180000E94B009249682E00E94F3235A924A9278
:10019000EAEEF2E0A42DB52D0E9447268FE00E94E2
:1001A000F7230E94610A22968FE00E94F32384E6DF
:1001B00090E00E9485245A924A9280E0A42DB52DA9
:1001C0008C9381E00E94F7235A924A9283E0A42DF7
:1001D000B52D8C9381E00E94F7230E94B0092496EC
:1001E00082E00E94F3235A924A92A42DB52DEAE5AB
:1001F000FDE40E949A248FE00E94F7230E94610A86
:1002000022968FE00E94F32384E690E00E948524EA
:100210005A924A9280E0A42DB52D8C9381E00E94E1
:10022000F7235A924A9284E0A42DB52D8C9381E055
:100230000E94F7230E94B009249682E00E94F323D3
:100240005A924A92A42DB52DEAE6FDE40E949A2422
:100250008EE00E94F7230E94610A22968EE00E949F
:10026000F3235A924A9280E0A42DB52D8C9381E01D
:100270000E94F7235A924A9285E0A42DB52D8C93C3
:1002800081E00E94F7230E94B009249682E00E9438
:10029000F3235A924A92A42DB52DEAE5FDE40E947B
:1002A0009A248FE00E94F7230E94610A22968FE031
:1002B0000E94F323E5E0F0E00E944E24DA9A959A3A
:1002C0000E941D095A924A9280E0A42DB52D8C936C
:1002D00081E00E94F7235A924A9282E0A42DB52D24
:1002E0008C9381E00E94F7230E94B009249682E05B
:1002F0000E94F3235A924A92A42DB52DE8E7FDE41B
:100300000E949A248FE00E94F7230E94610A22969D
:100310008FE00E94F32380E0809377025A924A9202
:1003200080E0A42DB52D8C9381E00E94F7235A9292
:100330004A9283E0A42DB52D8C9381E00E94F7238F
:100340000E94B009249682E00E94F3235A924A92B6
:10035000A42DB52DE8E8FDE40E949A248FE00E94C8
:10036000F7230E94610A22968FE00E94F3238EE019
:1003700091E00E9485245A924A9280917702A42D9E
:10038000B52D8C9381E00E94F7235A924A9283E024
:10039000A42DB52D8C9381E00E94F7230E94B00913
:1003A000249682E00E94F3235A924A92A42DB52DFE
:1003B000E8E9FDE40E949A2482E00E94F7230E946B
:1003C000610A229682E00E94F3238EE091E00E946F
:1003D00085245A924A9280917702A42DB52D8C9350
:1003E00081E00E94F7235A924A9283E0A42DB52D12
:1003F0008C9381E00E94F7230E94B009249682E04A
:100400000E94F3235A924A92A42DB52DEAE9FDE405
:100410000E949A2482E00E94F7230E94610A229699
:1004200082E00E94F3238EE091E00E9485245A929C
:100430004A9280917702A42DB52D8C9381E00E9481
:10044000F7235A924A9283E0A42DB52D8C9381E034
:100450000E94F7230E94B009249682E00E94F323B1
:100460005A924A92A42DB52DECE9FDE40E949A24FB
:1004700082E00E94F7230E94610A229682E00E9495
:10048000F3238EE091E00E9485245A924A92809153
:100490007702A42DB52D8C9381E00E94F7235A9208
:1004A0004A9283E0A42DB52D8C9381E00E94F7231E
:1004B0000E94B009249682E00E94F3235A924A9245
:1004C000A42DB52DEEE9FDE40E949A2482E00E945D
:1004D000F7230E94610A229682E00E94F3238EE0B5
:1004E00091E00E948524A7E7B2E08C918F5F8C9306
:1004F00000917702023011F00C94BB019598DA98C4
:100500005A924A9280E0A42DB52D8C9381E00E94EE
:10051000F7235A924A9282E0A42DB52D8C9381E064
:100520000E94F7230E94B009249682E00E94F323E0
:100530005A924A92A42DB52DE0EAFDE40E949A2435
:100540008FE00E94F7230E94610A22968FE00E94AA
:10055000F3235A924A9280917702A42DB52D8C9361
:1005600081E00E94F7235A924A9283E0A42DB52D90
:100570008C9381E00E94F7230E94B009249682E0C8
:100580000E94F3235A924A92A42DB52DE0EBFDE48C
:100590000E949A2482E00E94F7230E94610A229618
:1005A00082E00E94F3238EE091E00E9485245A921B
:1005B0004A9280917702A42DB52D8C9381E00E9400
:1005C000F7235A924A9283E0A42DB52D8C9381E0B3
:1005D0000E94F7230E94B009249682E00E94F32330
:1005E0005A924A92A42DB52DE8E9FDE40E949A247E
:1005F00082E00E94F7230E94610A229682E00E9414
:10060000F3238EE091E00E9485245A924A928091D1
:100610007702A42DB52D8C9381E00E94F7235A9286
:100620004A9283E0A42DB52D8C9381E00E94F7239C
:100630000E94B009249682E00E94F3235A924A92C3
:10064000A42DB52DEAE9FDE40E949A2482E00E94DF
:10065000F7230E94610A229682E00E94F3238EE033
:1006600091E00E9485245A924A9280917702A42DAB
:10067000B52D8C9381E00E94F7235A924A9283E031
:10068000A42DB52D8C9381E00E94F7230E94B00920
:10069000249682E00E94F3235A924A92A42DB52D0B
:1006A000ECE9FDE40E949A2482E00E94F7230E9474
:1006B000610A229682E00E94F3238EE091E00E947C
:1006C00085245A924A9280917702A42DB52D8C935D
:1006D00081E00E94F7235A924A9283E0A42DB52D1F
:1006E0008C9381E00E94F7230E94B009249682E057
:1006F0000E94F3235A924A92A42DB52DEEE9FDE40F
:100700000E949A2482E00E94F7230E94610A2296A6
:1007100082E00E94F3238EE091E00E948524A7E707
:10072000B2E08C918F5F8C9300917702063011F0CC
:100730000C94A9025A924A9280E0A42DB52D8C9374
:1007400081E00E94F7235A924A9282E0A42DB52DAF
:100750008C9381E00E94F7230E94B009249682E0E6
:100760000E94F3235A924A92A42DB52DE2EBFDE4A8
:100770000E949A248FE00E94F7230E94610A229629
:100780008FE00E94F323E2ECFDE40E9440240E94EB
:1007900047245A924A9280917702A42DB52D8C93CA
:1007A00081E00E94F7235A924A9283E0A42DB52D4E
:1007B0008C9381E00E94F7230E94B009249682E086
:1007C0000E94F3235A924A92A42DB52DE0EBFDE44A
:1007D0000E949A2482E00E94F7230E94610A2296D6
:1007E00082E00E94F3238EE091E00E948524E2ECF7
:1007F000FDE40E9440240E9447240E94C7155A929B
:100800004A9280917702A42DB52D8C9381E00E94AD
:10081000F7235A924A9283E0A42DB52D8C9381E060
:100820000E94F7230E94B009249682E00E94F323DD
:100830005A924A92A42DB52DE8E9FDE40E949A242B
:1008400082E00E94F7230E94610A229682E00E94C1
:10085000F3238EE091E00E9485245A924A9280917F
:100860007702A42DB52D8C9381E00E94F7235A9234
:100870004A9283E0A42DB52D8C9381E00E94F7234A
:100880000E94B009249682E00E94F3235A924A9271
:10089000A42DB52DEAE9FDE40E949A2482E00E948D
:1008A000F7230E94610A229682E00E94F3238EE0E1
:1008B00091E00E9485245A924A9280917702A42D59
:1008C000B52D8C9381E00E94F7235A924A9283E0DF
:1008D000A42DB52D8C9381E00E94F7230E94B009CE
:1008E000249682E00E94F3235A924A92A42DB52DB9
:1008F000ECE9FDE40E949A2482E00E94F7230E9422
:10090000610A229682E00E94F3238EE091E00E9429
:1009100085245A924A9280917702A42DB52D8C930A
:1009200081E00E94F7235A924A9283E0A42DB52DCC
:100930008C9381E00E94F7230E94B009249682E004
:100940000E94F3235A924A92A42DB52DEEE9FDE4BC
:100950000E949A2482E00E94F7230E94610A229654
:1009600082E00E94F3238EE091E00E948524A7E7B5
:10097000B2E08C918F5F8C935A924A9280E0A42DC2
:10098000B52D8C9381E00E94F7235A924A9282E01F
:10099000A42DB52D8C9381E00E94F7230E94B0090D
:1009A000249682E00E94F3235A924A92A42DB52DF8
:1009B000E6ECFDE40E949A248FE00E94F7230E9457
:1009C000610A22968FE00E94F3235A924A92809104
:1009D0007702A42DB52D8C9381E00E94F7235A92C3
:1009E0004A9283E0A42DB52D8C9381E00E94F723D9
:1009F0000E94B009249682E00E94F3235A924A9200
:100A0000A42DB52DE0EBFDE40E949A2482E00E9423
:100A1000F7230E94610A229682E00E94F3238EE06F
:100A200091E00E9485245A924A9280917702A42DE7
:100A3000B52D8C9381E00E94F7235A924A9283E06D
:100A4000A42DB52D8C9381E00E94F7230E94B0095C
:100A5000249682E00E94F3235A924A92A42DB52D47
:100A6000E8E9FDE40E949A2482E00E94F7230E94B4
:100A7000610A229682E00E94F3238EE091E00E94B8
:100A80008524E2ECFDE40E9440240E94472488E291
:100A900090E00E948524A2E3B2E0BA93AA930E9458
:100AA00089152296A2E3B2E0E6EDFDE40E948C26D1
:100AB00011F00C9441050E94C7155A924A928091F8
:100AC0007702A42DB52D8C9381E00E94F7235A92D2
:100AD0004A9283E0A42DB52D8C9381E00E94F723E8
:100AE0000E94B009249682E00E94F3235A924A920F
:100AF000A42DB52DEAE9FDE40E949A2482E00E942B
:100B0000F7230E94610A229682E00E94F3238EE07E
:100B100091E00E9485245A924A9280917702A42DF6
:100B2000B52D8C9381E00E94F7235A924A9283E07C
:100B3000A42DB52D8C9381E00E94F7230E94B0096B
:100B4000249682E00E94F3235A924A92A42DB52D56
:100B5000ECE9FDE40E949A2482E00E94F7230E94BF
:100B6000610A229682E00E94F3238EE091E00E94C7
:100B700085245A924A9280917702A42DB52D8C93A8
:100B800081E00E94F7235A924A9283E0A42DB52D6A
:100B90008C9381E00E94F7230E94B009249682E0A2
:100BA0000E94F3235A924A92A42DB52DEEE9FDE45A
:100BB0000E949A2482E00E94F7230E94610A2296F2
:100BC00082E00E94F3238EE091E00E948524A7E753
:100BD000B2E08C918F5F8C935A924A9280E0A42D60
:100BE000B52D8C9381E00E94F7235A924A9282E0BD
:100BF000A42DB52D8C9381E00E94F7230E94B009AB
:100C0000249682E00E94F3235A924A92A42DB52D95
:100C1000EAEDFDE40E949A248FE00E94F7230E94EF
:100C2000610A22968FE00E94F323EAEEFDE40E941F
:100C3000402482E20E944A24E4EFFDE40E94402422
:100C400082E20E944A240E9447245A924A9280914A
:100C50007702A42DB52D8C9381E00E94F7235A9240
:100C60004A9283E0A42DB52D8C9381E00E94F72356
:100C70000E94B009249682E00E94F3235A924A927D
:100C8000A42DB52DE0EBFDE40E949A2482E00E94A1
:100C9000F7230E94610A229682E00E94F3238EE0ED
:100CA00091E00E9485245A924A9280917702A42D65
:100CB000B52D8C9381E00E94F7235A924A9283E0EB
:100CC000A42DB52D8C9381E00E94F7230E94B009DA
:100CD000249682E00E94F3235A924A92A42DB52DC5
:100CE000E8E9FDE40E949A2482E00E94F7230E9432
:100CF000610A229682E00E94F323E5E0F0E00E9480
:100D00004E240E94C7158EE091E00E9485245A92DD
:100D10004A9280917702A42DB52D8C9381E00E9498
:100D2000F7235A924A9283E0A42DB52D8C9381E04B
:100D30000E94F7230E94B009249682E00E94F323C8
:100D40005A924A92A42DB52DEAE9FDE40E949A2414
:100D500082E00E94F7230E94610A229682E00E94AC
:100D6000F3238EE091E00E9485245A924A9280916A
:100D70007702A42DB52D8C9381E00E94F7235A921F
:100D80004A9283E0A42DB52D8C9381E00E94F72335
:100D90000E94B009249682E00E94F3235A924A925C
:100DA000A42DB52DECE9FDE40E949A2482E00E9476
:100DB000F7230E94610A229682E00E94F3238EE0CC
:100DC00091E00E9485245A924A9280917702A42D44
:100DD000B52D8C9381E00E94F7235A924A9283E0CA
:100DE000A42DB52D8C9381E00E94F7230E94B009B9
:100DF000249682E00E94F3235A924A92A42DB52DA4
:100E0000EEE9FDE40E949A2482E00E94F7230E940A
:100E1000610A229682E00E94F32384E690E00E9419
:100E200085245A924A9280917702A42DB52D8C93F5
:100E300081E00E94F7235A924A9283E0A42DB52DB7
:100E40008C9381E00E94F7230E94B009249682E0EF
:100E50000E94F323A7E7B2E08C918F5F8C935A92A4
:100E60004A9280917702A42DB52D8C9381E00E9447
:100E7000F7235A924A9283E0A42DB52D8C9381E0FA
:100E80000E94F7230E94B009249682E00E94F32377
:100E90005A924A92A42DB52DE0EBFDE40E949A24CB
:100EA00082E00E94F7230E94610A229682E00E945B
:100EB000F32382E390E00E9485245A924A92809123
:100EC0007702A42DB52D8C9381E00E94F7235A92CE
:100ED0004A9283E0A42DB52D8C9381E00E94F723E4
:100EE0000E94B009249682E00E94F3235A924A920B
:100EF000A42DB52DE8E9FDE40E949A2482E00E9429
:100F0000F7230E94610A229682E00E94F32382E383
:100F100090E00E9485245A924A9280917702A42DF3
:100F2000B52D8C9381E00E94F7235A924A9283E078
:100F3000A42DB52D8C9381E00E94F7230E94B00967
:100F4000249682E00E94F3235A924A92A42DB52D52
:100F5000EAE9FDE40E949A2482E00E94F7230E94BD
:100F6000610A229682E00E94F32382E390E00E94CD
:100F700085245A924A9280917702A42DB52D8C93A4
:100F800081E00E94F7235A924A9283E0A42DB52D66
:100F90008C9381E00E94F7230E94B009249682E09E
:100FA0000E94F3235A924A92A42DB52DECE9FDE458
:100FB0000E949A2482E00E94F7230E94610A2296EE
:100FC00082E00E94F32382E390E00E9485245A92FB
:100FD0004A9280917702A42DB52D8C9381E00E94D6
:100FE000F7235A924A9283E0A42DB52D8C9381E089
:100FF0000E94F7230E94B009249682E00E94F32306
:101000005A924A92A42DB52DEEE9FDE40E949A244D
:1010100082E00E94F7230E94610A229682E00E94E9
:10102000F32382E390E00E9485245A924A928091B1
:101030007702A42DB52D8C9381E00E94F7235A925C
:101040004A9283E0A42DB52D8C9381E00E94F72372
:101050000E94B009249682E00E94F3235A924A9299
:10106000A42DB52DECEFFDE40E949A2482E00E94AD
:10107000F7230E94610A229682E00E94F32382E312
:1010800090E00E948524A7E7B2E08C918F5F8C935B
:10109000009177020E3011F00C942F0780E08093BE
:1010A00077020E941D095A924A9280E0A42DB52D24
:1010B0008C9381E00E94F7235A924A9282E0A42DF9
:1010C000B52D8C9381E00E94F7230E94B0092496ED
:1010D00082E00E94F3235A924A92A42DB52DEEEF9E
:1010E000FDE40E949A248FE00E94F7230E94610A87
:1010F00022968FE00E94F3230E94C715DA9AEEE051
:10110000FEE40E9440240E94472482E390E00E9473
:101110008524E8E1FEE40E9440240E944724E3E0A5
:10112000F0E00E944E24DA980E94C7150E941D0923
:10113000DA9A0E9417200E94D7150E94C7220E94A7
:1011400045170E94A11B0E94211C0E94E01D0E94C5
:10115000FA190E947921DA98EAE0F0E00E944E2420
:101160000C949808F894FFCFDF98EF93FF93E4EE88
:10117000F3E00E945424FF91EF91DF9A0895DE98E6
:10118000DD985A924A9281E2A42DB52D8C9381E08C
:101190000E94F7230E949E09229681E00E94F32379
:1011A0005A924A9288ECA42DB52D8C9381E00E942E
:1011B000F7230E949E09229681E00E94F3235A920F
:1011C0004A9286E0A42DB52D8C9381E00E94F723EE
:1011D0000E949E09229681E00E94F3235A924A922D
:1011E00083E1A42DB52D8C9381E00E94F7230E940A
:1011F0009E09229681E00E94F3235A924A9280E24D
:10120000A42DB52D8C9381E00E94F7230E949E09A6
:10121000229681E00E94F3235A924A928CE0A42DF8
:10122000B52D8C9381E00E94F7230E949E0922969F
:1012300081E00E94F323DE9A089582E00E949424C4
:10124000DE98DD985A924A9280E2A42DB52D8C93B7
:1012500081E00E94F7230E949E09229681E00E946D
:10126000F3235A924A9280E8A42DB52D8C9381E005
:101270000E94F7230E949E09229681E00E94F32398
:101280005A924A9280E4A42DB52D8C9381E00E945D
:10129000F7230E949E09229681E00E94F323DD9AA3
:1012A00080E090E0A881B9818D939C93A881B98159
:1012B0000D911C91073F51E0150718F011F00C94A7
:1012C00077095A924A9280E0A42DB52D8C9381E043
:1012D0000E94F7230E94A709229681E00E94F3232F
:1012E000A881B9810E94FB2310F40C945609DE9A60
:1012F00082E0481A8827580A229608955A924A92FC
:101300008DE0A42DB52D8C9381E00E94F7230E94DF
:101310009E09229681E00E94F32308955A924A92F0
:101320008CE0A42DB52D8C9381E00E94F7230E94C0
:101330009E09229681E00E94F3230895DE98DD98AD
:1013400091E0A881B9810E945724DE9A0895DE9821
:10135000DD9A91E0A881B9810E945724DE9A089510
:1013600081E00E9494245A924A9280E2A42DB52DE5
:101370008C9381E00E94F7230E949E09229681E0CF
:101380000E94F323EF93FF93E4EEF3E00E945424D2
:10139000FF91EF91DE98DD98AC81BD810C9146E024
:1013A000049FA881B9810C92A881B9818C91805841
:1013B0008C9391E0A881B9810E945724AA81BB81B6
:1013C0000C9140E4040FA881B9810C9391E0A881AD
:1013D000B9810E945724DE9A81E0481A8827580A6A
:1013E0002296089582E00E94942481E00E94942431
:1013F000DE98DD985A924A9280E2A42DB52D8C9306
:1014000081E00E94F7230E949E09229681E00E94BB
:10141000F3235A924A9280E8A42DB52D8C9381E053
:101420000E94F7230E949E09229681E00E94F323E6
:101430005A924A9280E4A42DB52D8C9381E00E94AB
:10144000F7230E949E09229681E00E94F323DD9AF1
:1014500080E090E0AA81BB818D939C93AA81BB819F
:101460000D911C91073F51E0150718F011F00C94F5
:101470005A0A0E94F023A881B9810E94A0240C92EC
:101480000E94ED235A924A92AA81BB818C91A42D8D
:10149000B52D8C9381E00E94F7230E94A709229624
:1014A00081E00E94F323AA81BB810E94FB2310F4F8
:1014B0000C942E0ADE9A83E0481A8827580A24964C
:1014C000089581E00E94942482E00E94942481E0A7
:1014D0000E94942481E00E94942481E00E9494243C
:1014E000AA85BB850E948626A885B9858C9381E054
:1014F000AC81BD818C93A885B9854C91AC81BD81AF
:101500000C91041718F011F00C94E212AC81BD811B
:101510008C91EA85FB8501E00A93AF81B8850E9432
:101520004C26AE81BF81E2E2FEE40E948C2611F0DF
:101530000C94A00AE2EFF6E20E94ED230C949712BD
:10154000E4E2FEE40E948C2611F00C94AD0AE8EF70
:10155000F6E20E94ED230C949712E6E2FEE40E946C
:101560008C2611F00C94BA0AEEEFF6E20E94ED23FD
:101570000C949712E8E2FEE40E948C2611F00C9481
:10158000C70AE4E0F7E20E94ED230C949712EAE226
:10159000FEE40E948C2611F00C94D40AEAE0F7E2F3
:1015A0000E94ED230C949712ECE2FEE40E948C263C
:1015B00011F00C94E10AE0E1F7E20E94ED230C94B3
:1015C0009712EEE2FEE40E948C2611F00C94EE0AD3
:1015D000E6E1F7E20E94ED230C949712E0E3FEE4CB
:1015E0000E948C2611F00C94FB0AECE1F7E20E94B9
:1015F000ED230C949712E2E3FEE40E948C2611F096
:101600000C94080BE2E2F7E20E94ED230C9497128F
:10161000E4E3FEE40E948C2611F00C94150BE8E242
:10162000F7E20E94ED230C949712E6E3FEE40E9499
:101630008C2611F00C94220BEEE2F7E20E94ED23CF
:101640000C949712E8E3FEE40E948C2611F00C94AF
:101650002F0BE4E3F7E20E94ED230C949712EAE3E8
:10166000FEE40E948C2611F00C943C0BEAE3F7E2B6
:101670000E94ED230C949712ECE3FEE40E948C266A
:1016800011F00C94490BE0E4F7E20E94ED230C9476
:101690009712EEE3FEE40E948C2611F00C94560B98
:1016A000E6E4F7E20E94ED230C949712E0E4FEE4F6
:1016B0000E948C2611F00C94630BECE4F7E20E947C
:1016C000ED230C949712E2E4FEE40E948C2611F0C4
:1016D0000C94700BE2E5F7E20E94ED230C94971254
:1016E000E4E4FEE40E948C2611F00C947D0BE8E506
:1016F000F7E20E94ED230C949712E6E4FEE40E94C8
:101700008C2611F00C948A0BEEE5F7E20E94ED2393
:101710000C949712E8E4FEE40E948C2611F00C94DD
:10172000970BE4E6F7E20E94ED230C949712EAE4AB
:10173000FEE40E948C2611F00C94A40BEAE6F7E27A
:101740000E94ED230C949712ECE4FEE40E948C2698
:1017500011F00C94B10BE0E7F7E20E94ED230C943A
:101760009712EEE4FEE40E948C2611F00C94BE0B5E
:10177000E6E7F7E20E94ED230C949712E0E5FEE421
:101780000E948C2611F00C94CB0BECE7F7E20E9440
:10179000ED230C949712E2E5FEE40E948C2611F0F2
:1017A0000C94D80BE2E8F7E20E94ED230C94971218
:1017B000E4E5FEE40E948C2611F00C94E50BE8E8C9
:1017C000F7E20E94ED230C949712E6E5FEE40E94F6
:1017D0008C2611F00C94F20BEEE8F7E20E94ED2358
:1017E0000C949712E8E5FEE40E948C2611F00C940C
:1017F000FF0BE4E9F7E20E94ED230C949712EAE56F
:10180000FEE40E948C2611F00C940C0CEAE9F7E23D
:101810000E94ED230C949712ECE5FEE40E948C26C6
:1018200011F00C94190CE0EAF7E20E94ED230C94FD
:101830009712EEE5FEE40E948C2611F00C94260C23
:10184000E6EAF7E20E94ED230C949712E0E6FEE44C
:101850000E948C2611F00C94330CECEAF7E20E9403
:10186000ED230C949712E2E6FEE40E948C2611F020
:101870000C94400CE2EBF7E20E94ED230C949712DB
:10188000E4E6FEE40E948C2611F00C944D0CE8EB8B
:10189000F7E20E94ED230C949712E6E6FEE40E9424
:1018A0008C2611F00C945A0CEEEBF7E20E94ED231B
:1018B0000C949712E8E6FEE40E948C2611F00C943A
:1018C000670CE4ECF7E20E94ED230C949712EAE631
:1018D000FEE40E948C2611F00C94740CEAECF7E202
:1018E0000E94ED230C949712ECE6FEE40E948C26F5
:1018F00011F00C94810CE0EDF7E20E94ED230C94C2
:101900009712EEE6FEE40E948C2611F00C948E0CE9
:10191000E6EDF7E20E94ED230C949712E0E7FEE477
:101920000E948C2611F00C949B0CECEDF7E20E94C7
:10193000ED230C949712E2E7FEE40E948C2611F04E
:101940000C94A80CE2EEF7E20E94ED230C9497129F
:10195000E4E7FEE40E948C2611F00C94B50CE8EE4E
:10196000F7E20E94ED230C949712E6E7FEE40E9452
:101970008C2611F00C94C20CEEEEF7E20E94ED23DF
:101980000C949712E8E7FEE40E948C2611F00C9468
:10199000CF0CE4EFF7E20E94ED230C949712EAE7F4
:1019A000FEE40E948C2611F00C94DC0CEAEFF7E2C6
:1019B0000E94ED230C949712ECE7FEE40E948C2623
:1019C00011F00C94E90CE0E0F8E20E94ED230C9495
:1019D0009712EEE7FEE40E948C2611F00C94F60CB0
:1019E000E6E0F8E20E94ED230C949712E0E8FEE4B2
:1019F0000E948C2611F00C94030DECE0F8E20E949A
:101A0000ED230C949712E2E8FEE40E948C2611F07C
:101A10000C94100DE2E1F8E20E94ED230C94971271
:101A2000E4E8FEE40E948C2611F00C941D0DE8E120
:101A3000F8E20E94ED230C949712E6E8FEE40E947F
:101A40008C2611F00C942A0DEEE1F8E20E94ED23B1
:101A50000C949712E8E8FEE40E948C2611F00C9496
:101A6000370DE4E2F8E20E94ED230C949712EAE8C5
:101A7000FEE40E948C2611F00C94440DEAE2F8E298
:101A80000E94ED230C949712ECE8FEE40E948C2651
:101A900011F00C94510DE0E3F8E20E94ED230C9458
:101AA0009712EEE8FEE40E948C2611F00C945E0D75
:101AB000E6E3F8E20E94ED230C949712E0E9FEE4DD
:101AC0000E948C2611F00C946B0DECE3F8E20E945E
:101AD000ED230C949712E2E9FEE40E948C2611F0AB
:101AE0000C94780DE2E4F8E20E94ED230C94971236
:101AF000E4E9FEE40E948C2611F00C94850DE8E4E4
:101B0000F8E20E94ED230C949712E6E9FEE40E94AD
:101B10008C2611F00C94920DEEE4F8E20E94ED2375
:101B20000C949712E8E9FEE40E948C2611F00C94C4
:101B30009F0DE4E5F8E20E94ED230C949712EAE988
:101B4000FEE40E948C2611F00C94AC0DEAE5F8E25C
:101B50000E94ED230C949712ECE9FEE40E948C267F
:101B600011F00C94B90DE0E6F8E20E94ED230C941C
:101B70009712EEE9FEE40E948C2611F00C94C60D3B
:101B8000EEE2F7E20E94ED230C949712E0EAFEE405
:101B90000E948C2611F00C94D30DEAECF7E20E941F
:101BA000ED230C949712E2EAFEE40E948C2611F0D9
:101BB0000C94E00DE2EDF5E20E94ED230C949712F7
:101BC000E4EAFEE40E948C2611F00C94ED0DE8EDA1
:101BD000F5E20E94ED230C949712E6EAFEE40E94DF
:101BE0008C2611F00C94FA0DEEEDF5E20E94ED2337
:101BF0000C949712E8EAFEE40E948C2611F00C94F3
:101C0000070EE4EEF5E20E94ED230C949712EAEA47
:101C1000FEE40E948C2611F00C94140EEAEEF5E21C
:101C20000E94ED230C949712ECEAFEE40E948C26AD
:101C300011F00C94210EE0EFF5E20E94ED230C94DC
:101C40009712EEEAFEE40E948C2611F00C942E0E00
:101C5000E6EFF5E20E94ED230C949712E0EBFEE430
:101C60000E948C2611F00C943B0EECEFF5E20E94E2
:101C7000ED230C949712E2EBFEE40E948C2611F007
:101C80000C94480EE6E4F7E20E94ED230C949712C0
:101C9000E4EBFEE40E948C2611F00C94550EE2EE6B
:101CA000F7E20E94ED230C949712E6EBFEE40E940B
:101CB0008C2611F00C94620EE2E0F6E20E94ED2315
:101CC0000C949712E8EBFEE40E948C2611F00C9421
:101CD0006F0EE8E0F6E20E94ED230C949712EAEB17
:101CE000FEE40E948C2611F00C947C0EEEE0F6E2ED
:101CF0000E94ED230C949712ECEBFEE40E948C26DC
:101D000011F00C94890EE4E1F6E20E94ED230C94AC
:101D10009712EEEBFEE40E948C2611F00C94960EC6
:101D2000EAE1F6E20E94ED230C949712E0ECFEE467
:101D30000E948C2611F00C94A30EE0E2F6E20E94C1
:101D4000ED230C949712E2ECFEE40E948C2611F035
:101D50000C94B00EE6E2F6E20E94ED230C9497128A
:101D6000E4ECFEE40E948C2611F00C94BD0EECE233
:101D7000F6E20E94ED230C949712ECEFFDE40E9432
:101D80008C2611F00C94CA0EE2E3F6E20E94ED23D9
:101D90000C949712E6ECFEE40E948C2611F00C9451
:101DA000D70EE8E3F6E20E94ED230C949712E8ECDC
:101DB000FEE40E948C2611F00C94E40EEAE6F7E2B1
:101DC0000E94ED230C949712EAECFEE40E948C260C
:101DD00011F00C94F10EEEE3F6E20E94ED230C9468
:101DE0009712ECECFEE40E948C2611F00C94FE0E8F
:101DF000E4E4F6E20E94ED230C949712EEECFEE48C
:101E00000E948C2611F00C940B0FEAE4F6E20E947B
:101E1000ED230C949712E0EDFEE40E948C2611F065
:101E20000C94180FE6E7F7E20E94ED230C9497124A
:101E3000E2EDFEE40E948C2611F00C94250FE0E503
:101E4000F6E20E94ED230C949712E4EDFEE40E946A
:101E50008C2611F00C94320FE8E5F7E20E94ED2396
:101E60000C949712E6EDFEE40E948C2611F00C947F
:101E70003F0FE6E5F6E20E94ED230C949712E8EDA1
:101E8000FEE40E948C2611F00C944C0FE2E8F7E27D
:101E90000E94ED230C949712EAEDFEE40E948C263A
:101EA00011F00C94590FEEE1F8E20E94ED230C942E
:101EB0009712ECEDFEE40E948C2611F00C94660F54
:101EC000ECE5F6E20E94ED230C949712EEEDFEE4B1
:101ED0000E948C2611F00C94730FE2E6F6E20E9449
:101EE000ED230C949712E0EEFEE40E948C2611F094
:101EF0000C94800FE8E8F7E20E94ED230C9497120F
:101F0000E2EEFEE40E948C2611F00C948D0FE4E2C8
:101F1000F8E20E94ED230C949712E4EEFEE40E9496
:101F20008C2611F00C949A0FEAE3F7E20E94ED235D
:101F30000C949712E6EEFEE40E948C2611F00C94AD
:101F4000A70FE6EDF7E20E94ED230C949712E8EE5E
:101F5000FEE40E948C2611F00C94B40FE0EAF7E244
:101F60000E94ED230C949712EAEEFEE40E948C2668
:101F700011F00C94C10FE8E6F6E20E94ED230C94F8
:101F80009712ECEEFEE40E948C2611F00C94CE0F1A
:101F9000EEE6F6E20E94ED230C949712EEEEFEE4DC
:101FA0000E948C2611F00C94DB0FEAE5F8E20E9407
:101FB000ED230C949712E0EFFEE40E948C2611F0C2
:101FC0000C94E80FE8EBF7E20E94ED230C949712D3
:101FD000E2EFFEE40E948C2611F00C94F50FE4E58C
:101FE000F8E20E94ED230C949712EEE9FDE40E94C2
:101FF0008C2611F00C940210E4E7F6E20E94ED2327
:102000000C949712E4EFFEE40E948C2611F00C94DD
:102010000F10EAE7F6E20E94ED230C949712ECE928
:10202000FDE40E948C2611F00C941C10ECE8F6E202
:102030000E94ED230C949712E6EFFEE40E948C269A
:1020400011F00C942910E2E9F6E20E94ED230C94C1
:102050009712E8EFFEE40E948C2611F00C943610E3
:10206000E0E8F6E20E94ED230C949712EAEFFEE41A
:102070000E948C2611F00C944310E6E8F6E20E94D0
:10208000ED230C949712EAE9FDE40E948C2611F0EE
:102090000C945010E8E9F6E20E94ED230C9497129C
:1020A000ECEFFEE40E948C2611F00C945D10EEE93A
:1020B000F6E20E94ED230C949712E8E9FDE40E94F9
:1020C0008C2611F00C946A10E4EAF6E20E94ED23EB
:1020D0000C949712EEEFFEE40E948C2611F00C9403
:1020E0007710EAEAF6E20E94ED230C949712E0E002
:1020F000FFE40E948C2611F00C948410E0EDF7E2CE
:102100000E94ED230C949712E2E0FFE40E948C26DB
:1021100011F00C949110E0EBF6E20E94ED230C9488
:102120009712E0EBFDE40E948C2611F00C949E10B7
:10213000E6EBF6E20E94ED230C949712E4E0FFE454
:102140000E948C2611F00C94AB10ECEBF6E20E948E
:10215000ED230C949712E6E0FFE40E948C2611F028
:102160000C94B810E2ECF6E20E94ED230C94971266
:10217000E8E0FFE40E948C2611F00C94C510E8EC16
:10218000F6E20E94ED230C949712EAE0FFE40E942D
:102190008C2611F00C94D210EEECF6E20E94ED23A6
:1021A0000C949712ECE0FFE40E948C2611F00C9442
:1021B000DF10E4EDF6E20E94ED230C949712EEE0BE
:1021C000FFE40E948C2611F00C94EC10EAEDF6E28C
:1021D0000E94ED230C949712E0E1FFE40E948C260C
:1021E00011F00C94F910E0EEF6E20E94ED230C944D
:1021F0009712E2E1FFE40E948C2611F00C94061184
:10220000E6EEF6E20E94ED230C949712E4E1FFE47F
:102210000E948C2611F00C941311ECEEF6E20E9451
:10222000ED230C949712E6E1FFE40E948C2611F056
:102230000C942011E6E6F8E20E94ED230C9497122C
:10224000E8E1FFE40E948C2611F00C942D11E2E7E6
:10225000F8E20E94ED230C949712EAE1FFE40E9459
:102260008C2611F00C943A11ECE6F8E20E94ED2372
:102270000C949712ECE1FFE40E948C2611F00C9470
:102280004711E8E7F8E20E94ED230C949712EEE183
:10229000FFE40E948C2611F00C945411EEEAF8E24F
:1022A0000E94ED230C949712E0E2FFE40E948C263A
:1022B00011F00C946111EEE7F8E20E94ED230C940A
:1022C0009712E2E2FFE40E948C2611F00C946E114A
:1022D000E0ECF8E20E94ED230C949712E4E2FFE4B4
:1022E0000E948C2611F00C947B11E4EEF8E20E941F
:1022F000ED230C949712E6E2FFE40E948C2611F085
:102300000C948811EAEEF8E20E94ED230C949712E7
:10231000E8E2FFE40E948C2611F00C949511E8EAA3
:10232000F8E20E94ED230C949712EAE2FFE40E9487
:102330008C2611F00C94A211ECEFF8E20E94ED2330
:102340000C949712ECE2FFE40E948C2611F00C949E
:10235000AF11E8E0F9E20E94ED230C949712EEE24F
:10236000FFE40E948C2611F00C94BC11E8EDF8E219
:102370000E94ED230C949712E0E3FFE40E948C2668
:1023800011F00C94C911E4EBF8E20E94ED230C94D7
:102390009712E2E3FFE40E948C2611F00C94D61110
:1023A000E6ECF8E20E94ED230C949712E4E3FFE4DC
:1023B0000E948C2611F00C94E311E0E9F8E20E94EF
:1023C000ED230C949712E6E3FFE40E948C2611F0B3
:1023D0000C94F011E2EDF8E20E94ED230C949712B8
:1023E000E8E3FFE40E948C2611F00C94FD11E0EF6D
:1023F000F8E20E94ED230C949712EAE3FFE40E94B6
:102400008C2611F00C940A12E4E8F8E20E94ED2305
:102410000C949712ECE3FFE40E948C2611F00C94CC
:102420001712EEEDF8E20E94ED230C949712EEE302
:10243000FFE40E948C2611F00C942412E2E0F9E2F1
:102440000E94ED230C949712E0E4FFE40E948C2696
:1024500011F00C943112E6E9F8E20E94ED230C949D
:102460009712E2E4FFE40E948C2611F00C943E12D5
:10247000EAEBF8E20E94ED230C949712E9EFF2E008
:102480000E948E2611F00C944B12ECECF8E20E94A4
:10249000ED230C949712E4E4FFE40E948C2611F0E3
:1024A0000C945812E6EFF8E20E94ED230C94971278
:1024B000E6E4FFE40E948C2611F00C946512EAE831
:1024C000F8E20E94ED230C949712E8E4FFE40E94E6
:1024D0008C2611F00C947212E2EAF8E20E94ED23CD
:1024E0000C949712EAE4FFE40E948C2611F00C94FD
:1024F0007F12EEE0F9E20E94ED230C949712ECE4D7
:10250000FFE40E948C2611F00C948C12E4E1F9E2B5
:102510000E94ED230C949712EEE4FFE40E948C26B7
:1025200011F00C949712ECE9F8E20E94ED2381E09F
:10253000AA81BB818C93AA81BB810C91053018F0D4
:1025400011F00C94C5120E94F023A881B9810E9459
:10255000A0240C920E94ED235A924A92AA81BB8138
:102560008C91A42DB52D8C9381E00E94F7230E94BD
:10257000A709229681E00E94F323AA81BB818C9156
:102580008F5F8C9310F40C949B1280E0A881B9812A
:102590008C935A924A92AA81BB818C91A42DB52D1D
:1025A0008C9381E00E94F7230E94A709229681E084
:1025B0000E94F323AC81BD818C918F5F8C9310F4CA
:1025C0000C947B0ADE9A86E0481A8827580A2A96D5
:1025D00008957F49494931007C4A4A4931007F4981
:1025E000494936007C54542800007F010101030052
:1025F0007C0404040C00E0514F41FF00E0544C44C3
:10260000FC007C5554554400385554551800770843
:102610007F0877006C107C106C00414949493600F6
:102620004454545428007F1008047F007C20100874
:102630007C007F7F7F7F7F007842241278007C10AF
:102640002844000020413F017F0020443C047C00DE
:102650007C0810087C007C1010107C007F010101B8
:102660007F007C0404047C0004047C0404004728EC
:10267000100807007F7F7F7F7F000C1010107C0008
:102680000C127F120C0018247E2418007F7F7F7F9D
:1026900041007C404040FC007F7F7F4141007C4006
:1026A00078407C007F7F414141007C407840FC00C5
:1026B0007C50502000007F41414141004141414157
:1026C0004100414141417F007C5020007C0022417B
:1026D00049493E002844545438007F083E413E009A
:1026E0007C1038443800462919097F0008543414F6
:1026F0007C003E5149453E0000427F40000042615F
:10270000514946002241494936001814127F1000F1
:102710002745454539003E494949320061110905BF
:102720000300364949493600264949493E007E0999
:1027300009097E007F49494936003E414141220056
:102740007F4141413E007F49494941007F090909D4
:1027500001003E4149493A007F0808087F000041D6
:102760007F410000204141413F007F081422410089
:102770007F40404040007F0204027F007F04081039
:102780007F003E4141413E007F09090906003E416C
:1027900051617E007F0919294600064949493000E8
:1027A00001017F0101003F4040403F001F204020C9
:1027B0001F007F2010207F006314081463000304AF
:1027C0007804030061514945430020545454780073
:1027D0007F4844443800384444442800384444483E
:1027E0007F0038545454180000047E0500000C5239
:1027F000524A3C007F080404780000447D400000F9
:102800000040443D00007F201028440000417F40EC
:1028100000007C0418047C007C0804047800384420
:10282000444438007C1424241800182424147C0008
:102830007C0404080000085454542000043F444021
:1028400000003C4040407C001C2040201C003C40DC
:1028500030403C004428102844000C5050483C00B4
:102860004464544C4400000000000000006060001C
:1028700000000808080808000036360000000006BE
:1028800009090600007F414100000041417F00002E
:10289000552A552A550007097F0907004040404046
:1028A000400000563600000040400070700040407C
:1028B0000000000014141414140002015109060051
:1028C0007C7C0000000000005F00000000070007A3
:1028D0000000147F147F1400221408142200231314
:1028E000086462007C7C007F7F000005030000001C
:1028F000001C224100000041221C000014083E0878
:10290000140008083E0808000000503000002010A5
:10291000080402000204081020000000000000006B
:1029200000000000000000000080E0F8F8F8F0C0AF
:10293000000008081838F8F8F8F8F808080000004F
:102940000000000808F8F878180808000808D8F807
:10295000F8F8F8780808080818F8F8F0F0E000002F
:1029600000008888888888888888F800000000002F
:1029700000000000000000000000C0F03E0F010356
:102980000F3FFFFFFEF8E000000001071FFFFFFF01
:10299000FCF080000000C0F81F07010000000000EC
:1029A00080F8FFFFFF7F2760E0E0F0F8DC1F0F0FEB
:1029B0000701000000007844444444785048440033
:1029C00000000000000000008080C0E0F8FEC78129
:1029D0008101010101018187FFFFFFFFFCE0C08051
:1029E0008000031F7FFFFFFE7C0F030000000080BC
:1029F0008080C0F8FFFFFFFFCF80800001071F7FAE
:102A0000FFFFFCF0C080800000007C04080810205C
:102A100020407D00000000000000000000000000D9
:102A200000000808F8F8F8080000000000000000A6
:102A3000000000000000000000000000001818184E
:102A40000000000000000000000000000000000086
:102A500000000000000000000000000000003E2216
:102A60002222222222223E0000000000000000005C
:102A7000F8FCFE070181F1FFFF1F000078FCFE93C8
:102A800011190F8F46808E9E1F39F9F3E30301E180
:102A9000FFFF1F000000F8FCFE070301E1FEFF1F1F
:102AA000010181FFFF7F0602F1FFFF1E0000000011
:102AB00000009F909090909090909F0000000000E8
:102AC00000000000000101010100000101010100FE
:102AD00000000101010101000000010101010100EC
:102AE000000000000101010100000C1D1911191F57
:102AF0000F070100000001010100000000010101B9
:102B000001000000000010101010101010101F0025
:102B10000000A881B98188278C930E940F24A1E02E
:102B2000B1E08C9300910101003011F00C949A15E2
:102B30000C94C4150D3011F00C94A0150C94C41510
:102B40000A3011F00C94AF15A881B9818C918030B6
:102B500011F40C94AD150C94C6150C94C415009189
:102B600001010F3118F011F00C94B8150C94C41534
:102B7000A1E0B1E08C91A881B9818F930E940224D9
:102B80008F918D9388278C930C948D15089584E6EE
:102B900090E00E9485240E940F24A1E0B1E08C9374
:102BA00000910101003011F00C94CB1508950E94A2
:102BB0000924A2E0B1E08C9300910201013011F0F0
:102BC0000C944417A2E3B2E0BA93AA930E94891529
:102BD0002296E2E3F2E004E0A3E0B1E00E94532693
:102BE000A3E0B1E0E0E5FFE40E948C2611F00C9434
:102BF0003E17A2E3B2E00E948626EA2FFB2F33970E
:102C0000F0400FEFA3E1B1E00E945326E3E1F1E0D1
:102C100001E0A6E1B1E00E945326A6E1B1E0ECE2BA
:102C2000FFE40E948C2611F00C942316A2E3B2E07C
:102C30000E948626EA2FFB2F3297F0400FEFA3E188
:102C4000B1E00E945326E1E0F0E00E944E24AFE99B
:102C5000B0E088278C93E6E5FFE40E944024A3E1DE
:102C6000B1E00E943A240E9447248AE090E00E944A
:102C70008524A2E3B2E0BA93AA930E948915229612
:102C80008AE090E00E948524A2E3B2E0BA93AA937E
:102C90000E948915229686E1E2E3F2E00CE00A93B5
:102CA000AFE9B0E00E944C26E2E3F2E0A8E1B1E037
:102CB0000E9447268AE090E00E948524A2E3B2E0C9
:102CC000BA93AA930E9489152296E2E3F2E0A8E162
:102CD000B1E00E944726E8E1F1E00EE0A8E1B1E0B2
:102CE0000E945326DA9884E690E00E948524DA9ABE
:102CF00082E390E00E948524A7E7B2E08C918F5F89
:102D00008C93009177020A3011F00C94721680E0D7
:102D1000809377025A924A9280E0A42DB52D8C932D
:102D200081E00E94F7235A924A9282E0A42DB52DA9
:102D30008C9381E00E94F7230E94B009249682E0E0
:102D40000E94F3235A924A92A42DB52DE0E6FFE4A7
:102D50000E949A248FE00E94F7230E94610A229623
:102D60008FE00E94F3235A924A9280E0A42DB52D61
:102D70008C9381E00E94F7235A924A9282E0A42D1C
:102D8000B52D8C9381E00E94F7230E94B009249610
:102D900082E00E94F3235A924A92EFE9F0E0A42DD8
:102DA000B52D0E9447268CE00E94F7230E94610AFD
:102DB00022968CE00E94F3235A924A9280E0A42D3E
:102DC000B52D8C9381E00E94F7235A924A9283E0BA
:102DD000A42DB52D8C9381E00E94F7230E94B009A9
:102DE000249682E00E94F3235A924A92A42DB52D94
:102DF000E0E6FFE40E949A248FE00E94F7230E94FD
:102E0000610A22968FE00E94F3235A924A9280E050
:102E1000A42DB52D8C9381E00E94F7235A924A92FB
:102E200083E0A42DB52D8C9381E00E94F7230E94AE
:102E3000B009249682E00E94F3235A924A92E8E174
:102E4000F1E0A42DB52D0E94472689E70E94F723C3
:102E50000E94610A229689E70E94F323EAEEFDE4CC
:102E60000E94402482E20E944A24E4EFFDE40E9492
:102E7000402482E20E944A240E94472484E690E093
:102E80000E9485240E94C7150895A8E1B1E0E2E2FE
:102E9000FEE40E948C2611F00C9488179698929864
:102EA00080917A028F7780937A02ABE7B2E0E0E715
:102EB000FFE40E949A24A8E1B1E088278C935A92FB
:102EC0004A9280E0A42DB52D8C9381E00E94F723D7
:102ED0005A924A9283E0A42DB52D8C9381E00E94F2
:102EE000F7230E94B009249682E00E94F3235A92AD
:102EF0004A92A42DB52DE4E7FFE40E949A248FE0C6
:102F00000E94F7230E94610A22968FE00E94F32319
:102F1000A8E1B1E0E4E2FEE40E948C2611F00C94FA
:102F2000CF17969AE8E2F0E00E944E24929A8091A0
:102F30007A02806880937A02ABE7B2E0E4E8FFE4CB
:102F40000E949A24A8E1B1E088278C935A924A9271
:102F500080E0A42DB52D8C9381E00E94F7235A9236
:102F60004A9283E0A42DB52D8C9381E00E94F72333
:102F70000E94B009249682E00E94F3235A924A925A
:102F8000A42DB52DE8E8FFE40E949A248FE00E946A
:102F9000F7230E94610A22968FE00E94F323A8E1A2
:102FA000B1E0E6E2FEE40E948C2611F00C943418A5
:102FB0000E94B51EA8E1B1E088278C93AFE9B0E08C
:102FC00088278C935A924A9280E0A42DB52D8C9339
:102FD00081E00E94F7235A924A9282E0A42DB52DF7
:102FE0008C9381E00E94F7230E94B009249682E02E
:102FF0000E94F3235A924A92A42DB52DE0E6FFE4F5
:103000000E949A248FE00E94F7230E94610A229670
:103010008FE00E94F3235A924A9280E0A42DB52DAE
:103020008C9381E00E94F7235A924A9283E0A42D68
:10303000B52D8C9381E00E94F7230E94B00924965D
:1030400082E00E94F3235A924A92A42DB52DE0E625
:10305000FFE40E949A248FE00E94F7230E94610AF5
:1030600022968FE00E94F323A8E1B1E0E8E2FEE4BB
:103070000E948C2611F00C9499180E94721FA8E1EE
:10308000B1E088278C93AFE9B0E088278C935A92FF
:103090004A9280E0A42DB52D8C9381E00E94F72305
:1030A0005A924A9282E0A42DB52D8C9381E00E9421
:1030B000F7230E94B009249682E00E94F3235A92DB
:1030C0004A92A42DB52DE0E6FFE40E949A248FE0F9
:1030D0000E94F7230E94610A22968FE00E94F32348
:1030E0005A924A9280E0A42DB52D8C9381E00E94E3
:1030F000F7235A924A9283E0A42DB52D8C9381E058
:103100000E94F7230E94B009249682E00E94F323D4
:103110005A924A92A42DB52DE0E6FFE40E949A242B
:103120008FE00E94F7230E94610A22968FE00E949E
:10313000F323A8E1B1E0EAE2FEE40E948C2611F05C
:103140000C94B6180E94FA19E6E8F2E0A1E9B1E0A1
:103150000E944726E0E9F2E0A1E9B1E00E940224E2
:103160000E9447260E94B8190E94C715A8E1B1E045
:10317000ECE2FEE40E948C2611F00C94C8188091B9
:103180007A028F7B80937A02A8E1B1E088278C9342
:10319000A8E1B1E0EEE2FEE40E948C2611F00C946E
:1031A000DA1880917A02806480937A02A8E1B1E013
:1031B00088278C93A8E1B1E0E0E3FEE40E948C262E
:1031C00011F00C94ED18E8E9FFE40E9440240E94FD
:1031D0004724A8E1B1E088278C93A8E1B1E0E2E3BD
:1031E000FEE40E948C2611F00C940019E0EAFFE442
:1031F0000E9440240E944724A8E1B1E088278C93D4
:10320000A8E1B1E0E8EAFFE40E948C2611F00C94FA
:103210003219EFE9F0E0ADEDB2E00E944726E0E0C0
:10322000F0E0ADEDB2E07BE70E946126A1E9B1E0FC
:10323000E4EBFFE40E949A24EDEDF2E0A1E9B1E0B5
:103240000E9402240E944726A1E9B1E00E940224C4
:10325000EEEBFFE40E949A240E94B819A8E1B1E0C5
:1032600088278C93A8E1B1E0E2E4FFE40E948C2679
:1032700011F00C94B719A1E9B1E0E2ECFFE40E946F
:103280009A248AE0A1E9B1E08F930E9402248F91F1
:103290008D9388278C93A1E9B1E00E940224EAEC87
:1032A000FFE40E949A24E6E8F2E0A1E9B1E00E947E
:1032B00002240E944726E0E9F2E0A1E9B1E00E9481
:1032C00002240E9447268AE0A1E9B1E08F930E9480
:1032D00002248F918D9388278C93A1E9B1E00E94FD
:1032E0000224E0EDFFE40E949A24EBE7F2E0A1E97A
:1032F000B1E00E9402240E9447268AE0A1E9B1E0E1
:103300008F930E9402248F918D9388278C93A1E93B
:10331000B1E00E940224E6EDFFE40E949A24EFE768
:10332000F2E0A1E9B1E00E9402240E9447268AE06F
:10333000A1E9B1E08F930E9402248F918D93882799
:103340008C93A1E9B1E00E940224E2EEFFE40E9426
:103350009A24E1E8F2E0A1E9B1E00E9402240E948F
:1033600047260E94B819A8E1B1E088278C930895F8
:10337000EAEFFFE40E94402482E20E944A24ADED7D
:10338000B2E00E943A2482E20E944A240E9447242A
:1033900088EC90E00E948524A1E9B1E00E943A24E3
:1033A0008AE10E944A240E9447248AE10E944A241A
:1033B000E1E0F0E00E944E248DE00E944A240E9449
:1033C0004724DA9884E690E00E948524DA9A82E322
:1033D00090E00E948524A7E7B2E08C918F5F8C93E8
:1033E000009177020A3011F00C94E11980E080938B
:1033F0007702089583E0E0E30E94FB24002762FA4D
:103400000EF401E041E0041711F00C943C1A8FEF28
:1034100080938502A6E8B2E0E4E0F0E50E949A24F9
:103420005A924A9280E0A42DB52D8C9381E00E949F
:10343000F7235A924A9281E0A42DB52D8C9381E016
:103440000E94F7230E94B009249682E00E94F32391
:103450005A924A92E6E8F2E0A42DB52D0E94472642
:1034600086E00E94F7230E94610A229686E00E946D
:10347000F32308950C94E61A6CEC83E0E0E3BB2799
:10348000A6E121E02A930E942E2564E483E0E0E394
:10349000BB27A6E121E02A930E942E258EEE92E022
:1034A0000E94852483E0E0E30E94FB246CEC83E02F
:1034B000E0E3BB27A6E121E02A930E942E256EEBD4
:1034C00083E0E0E3BB27A6E121E02A930E942E25BA
:1034D000BB27A6E183E0E0E321E02A930E94582580
:1034E000ACE8B2E05C93BB27A6E183E0E0E321E037
:1034F0002A930E945825ADE8B2E05C9300918D02BA
:10350000083F18F011F00C94871A0C949D1A0FEFD5
:1035100040918C02041BACE8B2E00C930FEF409199
:103520008D02041BADE8B2E00C93A6E8B2E0E8E13E
:10353000FFE40E949A240C94A31AA6E8B2E0EEE3FA
:10354000FFE40E949A2400918C0240E10E947626BA
:10355000AEE8B2E00C9300918D0240E1049FAFE829
:10356000B2E00C9200918E0240918F02040FA5E808
:10357000B2E00C93A6E8B2E0E8E1FFE40E948C26FA
:1035800011F00C94CA1A00918E0241E0040FA5E8D4
:10359000B2E00C93A6E8B2E0EEE3FFE40E948C26D2
:1035A00081E009F080E08F9300918502003081E096
:1035B00009F080E09F918923882311F40C94E61A86
:1035C000A6E8B2E0E6E1FFE40E949A24A0E9B2E0B6
:1035D000E5E8F2E00E94CB25E0E9F2E0ACE7B7E0F5
:1035E0000E944726ECE7F7E0A0E9B2E01127222786
:1035F00000E033270E94AE245A924A9280E0A42D24
:10360000B52D8C9381E00E94F7235A924A9281E073
:10361000A42DB52D8C9381E00E94F7230E94B00960
:10362000249682E00E94F3235A924A92A42DB52D4B
:10363000E0E6FFE40E949A248FE00E94F7230E94B4
:10364000610A22968FE00E94F3235A924A9280E008
:10365000A42DB52D8C9381E00E94F7235A924A92B3
:1036600081E0A42DB52D8C9381E00E94F7230E9468
:10367000B009249682E00E94F3235A924A92E6E827
:10368000F2E0A42DB52D0E94472686E00E94F72384
:103690000E94610A229686E00E94F3235A924A927F
:1036A00081E0A42DB52D8C9381E00E94F7235A92DE
:1036B0004A9281E0A42DB52D8C9381E00E94F723DE
:1036C0000E94B009249682E00E94F3235A924A9203
:1036D000E0E9F2E0A42DB52D0E94472685E00E9486
:1036E000F7230E94610A229685E00E94F3235A92F2
:1036F0004A9283E0A42DB52D8C9381E00E94F7239C
:103700005A924A9281E0A42DB52D8C9381E00E94BB
:10371000F7230E94B009249682E00E94F3235A9274
:103720004A92A42DB52DEAE0F0E50E949A2483E0A8
:103730000E94F7230E94610A229683E00E94F323ED
:103740000895EEE0F0E50E9440240E94472484EFB3
:1037500091E00E948524A2E3B2E0BA93AA930E946A
:103760008915229684E690E00E948524A2E3B2E0C7
:10377000BA93AA930E9489152296E2E3F2E0AEE999
:10378000B2E00E9447268CE0EEE9F2E009E00A93FD
:10379000AEE9B2E00E944C265A924A9280E0A42DF3
:1037A000B52D8C9381E00E94F7235A924A9280E0D3
:1037B000A42DB52D8C9381E00E94F7230E94B009BF
:1037C000249682E00E94F3235A924A92A42DB52DAA
:1037D000E8E1F0E50E949A248CE00E94F7230E9421
:1037E000610A22968CE00E94F3235A924A9280E06A
:1037F000A42DB52D8C9381E00E94F7235A924A9212
:1038000080E0A42DB52D8C9381E00E94F7230E94C7
:10381000B009249682E00E94F3235A924A92EEE97C
:10382000F2E0A42DB52D0E94472685E10E94F723E2
:103830000E94610A229685E10E94F3230E94C71527
:1038400008955A924A928BE0A42DB52D8C9381E075
:103850000E94F7235A924A9280E0A42DB52D8C93B2
:1038600081E00E94F7230E94B009249682E00E9422
:10387000F3235A924A92A42DB52DE0E4FFE40E946E
:103880009A2482E00E94F7230E94610A229682E035
:103890000E94F323E4E2F0E50E9440240E944724C2
:1038A0008CE291E00E948524A2E3B2E0BA93AA934D
:1038B0000E948915229684E690E00E948524A2E366
:1038C000B2E0BA93AA930E9489152296E2E3F2E04D
:1038D000A6E9B2E00E94472687E0E6E9F2E002E0CE
:1038E0000A93A6E9B2E00E944C26A6E9B2E00E9443
:1038F0001526ADE9B2E00C935A924A928CE0A42DC1
:10390000B52D8C9381E00E94F7235A924A9280E071
:10391000A42DB52D8C9381E00E94F7230E94B0095D
:10392000249682E00E94F3235A924A92A42DB52D48
:10393000ECE2F0E50E949A2483E00E94F7230E94C3
:10394000610A229683E00E94F32300919D020030D9
:1039500080E010F009F081E08F9300919D02043027
:1039600081E008F080E09F918923882311F40C9472
:10397000E41C5A924A928CE0A42DB52D8C9381E0E0
:103980000E94F7235A924A9280E0A42DB52D8C9381
:1039900081E00E94F7230E94B009249682E00E94F1
:1039A000F3235A924A92A42DB52DE0E3F0E50E944C
:1039B0009A2483E00E94F7230E94610A229683E002
:1039C0000E94F3230C94DD1D00919D02043080E0E1
:1039D00010F009F081E08F9300919D02093081E0A1
:1039E00008F080E09F918923882311F40C94231D13
:1039F0005A924A928CE0A42DB52D8C9381E00E94BE
:103A0000F7235A924A9280E0A42DB52D8C9381E041
:103A10000E94F7230E94B009249682E00E94F323BB
:103A20005A924A92A42DB52DE4E3F0E50E949A241F
:103A300083E00E94F7230E94610A229683E00E949D
:103A4000F3230C94DD1D00919D02093080E010F0FD
:103A500009F081E08F9300919D020F3081E008F022
:103A600080E09F918923882311F40C94621D5A925F
:103A70004A928CE0A42DB52D8C9381E00E94F7230F
:103A80005A924A9280E0A42DB52D8C9381E00E9439
:103A9000F7230E94B009249682E00E94F3235A92F1
:103AA0004A92A42DB52DE8E3F0E50E949A2483E024
:103AB0000E94F7230E94610A229683E00E94F3236A
:103AC0000C94DD1D00919D020F3080E010F009F094
:103AD00081E08F9300919D02003281E008F080E048
:103AE0009F918923882311F40C94A11D5A924A9224
:103AF0008CE0A42DB52D8C9381E00E94F7235A927F
:103B00004A9280E0A42DB52D8C9381E00E94F7238A
:103B10000E94B009249682E00E94F3235A924A92AE
:103B2000A42DB52DECE3F0E50E949A2483E00E94D9
:103B3000F7230E94610A229683E00E94F3230C94EB
:103B4000DD1D00919D02003081E009F080E08F933F
:103B500000919D02033681E009F080E09F91892B5E
:103B6000882311F40C94DD1D5A924A928CE0A42D06
:103B7000B52D8C9381E00E94F7235A924A9280E0FF
:103B8000A42DB52D8C9381E00E94F7230E94B009EB
:103B9000249682E00E94F3235A924A92A42DB52DD6
:103BA000EEE2FFE40E949A2482E00E94F7230E9442
:103BB000610A229682E00E94F3230E94C7150895AD
:103BC000E0E4F0E50E9440240E94472480E991E06F
:103BD0000E948524A2E3B2E0BA93AA930E948915B9
:103BE000229680E991E00E948524A2E3B2E0BA9394
:103BF000AA930E948915229689E0E2E3F2E008E0A8
:103C00000A93A3EBB2E00E944C265A924A9280E0BB
:103C1000A42DB52D8C9381E00E94F7235A924A92ED
:103C200085E0A42DB52D8C9381E00E94F7230E949E
:103C3000B009249682E00E94F3235A924A92A42D5E
:103C4000B52DE0E6FFE40E949A248FE00E94F7235E
:103C50000E94610A22968FE00E94F3235A924A92B0
:103C600080E0A42DB52D8C9381E00E94F7235A9219
:103C70004A9285E0A42DB52D8C9381E00E94F72314
:103C80000E94B009249682E00E94F3235A924A923D
:103C9000E3EBF2E0A42DB52D0E94472685E10E94BA
:103CA000F7230E94610A229685E10E94F32382E1B4
:103CB000E2E3F2E005E00A93A8ECB2E00E944C26B1
:103CC0005A924A9280E0A42DB52D8C9381E00E94F7
:103CD000F7235A924A9284E0A42DB52D8C9381E06B
:103CE0000E94F7230E94B009249682E00E94F323E9
:103CF0005A924A92A42DB52DE0E6FFE40E949A2440
:103D00008FE00E94F7230E94610A22968FE00E94B2
:103D1000F3235A924A9280E0A42DB52D8C9381E032
:103D20000E94F7235A924A9284E0A42DB52D8C93D9
:103D300081E00E94F7230E94B009249682E00E944D
:103D4000F3235A924A92E8ECF2E0A42DB52D0E949A
:103D5000472685E10E94F7230E94610A229685E1A9
:103D60000E94F3230E94C7150895EAE4F0E50E943B
:103D70004024ADEDB2E00E943A24E8E4FFE40E9462
:103D800040240E94472484E690E00E9485245A92B1
:103D90004A9280E0A42DB52D8C9381E00E94F723F8
:103DA0005A924A9282E0A42DB52D8C9381E00E9414
:103DB000F7230E94B009249682E00E94F3235A92CE
:103DC0004A92A42DB52DE0E6FFE40E949A248FE0EC
:103DD0000E94F7230E94610A22968FE00E94F3233B
:103DE0005A924A9280E0A42DB52D8C9381E00E94D6
:103DF000F7235A924A9282E0A42DB52D8C9381E04C
:103E00000E94F7230E94B009249682E00E94F323C7
:103E10005A924A92A42DB52DEEE4F0E50E949A2420
:103E20008AE00E94F7230E94610A22968AE00E949B
:103E3000F3235A924A9280E0A42DB52D8C9381E011
:103E40000E94F7235A924A9283E0A42DB52D8C93B9
:103E500081E00E94F7230E94B009249682E00E942C
:103E6000F3235A924A92A42DB52DE0E6FFE40E9476
:103E70009A248FE00E94F7230E94610A22968FE025
:103E80000E94F3235A924A9280E0A42DB52D8C9380
:103E900081E00E94F7235A924A9283E0A42DB52D27
:103EA0008C9381E00E94F7230E94B009249682E05F
:103EB0000E94F3235A924A92EDEDF2E0A42DB52D23
:103EC0000E9447268DE00E94F7230E94610A2296F5
:103ED0008DE00E94F323E4E1F0E00E944E240E9472
:103EE000C71508955A924A9280E0A42DB52D8C935F
:103EF00081E00E94F7235A924A9282E0A42DB52DC8
:103F00008C9381E00E94F7230E94B009249682E0FE
:103F10000E94F3235A924A92A42DB52DE0E6FFE4C5
:103F20000E949A248FE00E94F7230E94610A229641
:103F30008FE00E94F3235A924A9280E0A42DB52D7F
:103F40008C9381E00E94F7235A924A9282E0A42D3A
:103F5000B52D8C9381E00E94F7230E94B00924962E
:103F600082E00E94F3235A924A92A42DB52DE8E5EF
:103F7000F0E50E949A248FE00E94F7230E94610AD4
:103F800022968FE00E94F3235A924A9280E0A42D59
:103F9000B52D8C9381E00E94F7235A924A9283E0D8
:103FA000A42DB52D8C9381E00E94F7230E94B009C7
:103FB000249682E00E94F3235A924A92A42DB52DB2
:103FC000E0E6FFE40E949A248FE00E94F7230E941B
:103FD000610A22968FE00E94F323E8E6F0E50E9452
:103FE00040240E944724E1E0F0E00E944E24A2E336
:103FF000B2E0BA93AA930E9489152296A2E3B2E096
:10400000BA93AA930E9489152296A2E3B2E0BA93CA
:10401000AA930E9489152296E2E3F2E0A1E9B1E0B9
:104020000E9447260E94B8190E94C71508955A9207
:104030004A9280E0A42DB52D8C9381E00E94F72355
:104040005A924A9283E0A42DB52D8C9381E00E9470
:10405000F7230E94B009249682E00E94F3235A922B
:104060004A92A42DB52DE0E6FFE40E949A248FE049
:104070000E94F7230E94610A22968FE00E94F32398
:104080000027AAE7B2E08C9187FB0EF401E040E044
:10409000041711F00C947D205A924A9280E0A42DCE
:1040A000B52D8C9381E00E94F7235A924A9283E0C7
:1040B000A42DB52D8C9381E00E94F7230E94B009B6
:1040C000249682E00E94F3235A924A92A42DB52DA1
:1040D000E4E7FFE40E949A248FE00E94F7230E9405
:1040E000610A22968FE00E94F323ABE7B2E0E0E79B
:1040F000FFE40E949A240C94AC205A924A9280E0E9
:10410000A42DB52D8C9381E00E94F7235A924A92F8
:1041100083E0A42DB52D8C9381E00E94F7230E94AB
:10412000B009249682E00E94F3235A924A92A42D69
:10413000B52DE8E8FFE40E949A248FE00E94F7235F
:104140000E94610A22968FE00E94F323ABE7B2E05F
:10415000E4E8FFE40E949A240027A0E3B0E08C91F9
:1041600084FB0EF401E040E0041711F00C940C21E4
:104170005A924A9280E0A42DB52D8C9381E00E9442
:10418000F7235A924A9282E0A42DB52D8C9381E0B8
:104190000E94F7230E94B009249682E00E94F32334
:1041A0005A924A92A42DB52DE0E6FFE40E949A248B
:1041B0008FE00E94F7230E94610A22968FE00E94FE
:1041C000F3235A924A9280E0A42DB52D8C9381E07E
:1041D0000E94F7235A924A9282E0A42DB52D8C9327
:1041E00081E00E94F7230E94B009249682E00E9499
:1041F000F3235A924A92A42DB52DE2E7F0E50E94EE
:104200009A248FE00E94F7230E94610A22968FE091
:104210000E94F3230C9472215A924A9280E0A42DBA
:10422000B52D8C9381E00E94F7235A924A9282E046
:10423000A42DB52D8C9381E00E94F7230E94B00934
:10424000249682E00E94F3235A924A92A42DB52D1F
:10425000E0E6FFE40E949A248FE00E94F7230E9488
:10426000610A22968FE00E94F3235A924A9280E0DC
:10427000A42DB52D8C9381E00E94F7235A924A9287
:1042800082E0A42DB52D8C9381E00E94F7230E943B
:10429000B009249682E00E94F3235A924A92A42DF8
:1042A000B52DE2E8F0E50E949A248CE00E94F72305
:1042B0000E94610A22968CE00E94F323E2E0F0E083
:1042C0000E944E240027A0E3B0E08C9184FB0EF402
:1042D00001E041E0041711F00C9472210C947F006E
:1042E0000C9472210E94C7158AE090E00E948524F8
:1042F00008950027A0E3B0E08C9187FB0EF401E065
:1043000041E0041711F00C9425225A924A9286E05B
:10431000A42DB52D8C9381E00E94F7235A924A92E6
:1043200081E0A42DB52D8C9381E00E94F7230E949B
:10433000B009249682E00E94F3235A924A92A42D57
:10434000B52DEEE8F0E50E949A2489E00E94F7235B
:104350000E94610A229689E00E94F323AFE7B2E04F
:10436000E4E2FEE40E949A24E1E0F0E00E944E24A0
:104370000027AAE7B2E08C9186FB0EF401E040E052
:10438000041711F00C942322A1E9B1E0E8E9F0E56B
:104390000E949A245A924A9280E0A42DB52D8C93C3
:1043A00081E00E94F7235A924A9281E0A42DB52D14
:1043B0008C9381E00E94F7230E94B009249682E04A
:1043C0000E94F3235A924A92A42DB52DE0E6FFE411
:1043D0000E949A248FE00E94F7230E94610A22968D
:1043E0008FE00E94F3235A924A9280E0A42DB52DCB
:1043F0008C9381E00E94F7235A924A9281E0A42D87
:10440000B52D8C9381E00E94F7230E94B009249679
:1044100082E00E94F3235A924A92A42DB52DE0EA3D
:10442000F0E50E949A248FE00E94F7230E94610A1F
:1044300022968FE00E94F3230E94B81980917A029D
:10444000806480937A020C9454225A924A9286E0B5
:10445000A42DB52D8C9381E00E94F7235A924A92A5
:1044600081E0A42DB52D8C9381E00E94F7230E945A
:10447000B009249682E00E94F3235A924A92A42D16
:10448000B52DE0EBF0E50E949A2489E00E94F72325
:104490000E94610A229689E00E94F323AFE7B2E00E
:1044A000E2E2FEE40E949A240027AAE7B2E08C919F
:1044B00086FB0EF401E040E0041711F00C94912209
:1044C0005A924A928DE0A42DB52D8C9381E00E94E2
:1044D000F7235A924A9281E0A42DB52D8C9381E066
:1044E0000E94F7230E94B009249682E00E94F323E1
:1044F0005A924A92A42DB52DE6E1FFE40E949A2437
:1045000082E00E94F7230E94610A229682E00E94C4
:10451000F323A1E8B2E0EAEBF0E50E949A240C94C0
:10452000C0225A924A928DE0A42DB52D8C9381E041
:104530000E94F7235A924A9281E0A42DB52D8C93C4
:1045400081E00E94F7230E94B009249682E00E9435
:10455000F3235A924A92A42DB52DE2E3FFE40E9480
:104560009A2482E00E94F7230E94610A229682E048
:104570000E94F323A1E8B2E0EEEBF0E50E949A245A
:104580000E94C7158AE090E00E9485240895E2EC1D
:10459000F0E50E9440240E9447248AE090E00E94B7
:1045A0008524A2E3B2E0BA93AA930E9489152296C9
:1045B0008AE090E00E948524A2E3B2E0BA93AA9335
:1045C0000E948915229686E1E2E3F2E00CE00A936C
:1045D000AFE9B0E00E944C26E2E3F2E0A8E1B1E0EE
:1045E0000E944726E8E1F1E004E0A8E1B1E00E9482
:1045F0005326A8E1B1E0ECECF0E50E948C2611F026
:104600000C94E6238AE090E00E948524A2E3B2E0C5
:10461000BA93AA930E9489152296E2E3F2E0A8E1F8
:10462000B1E00E944726E8E1F1E00EE0A8E1B1E048
:104630000E945326DA9884E690E00E948524DA9A54
:1046400082E390E00E948524A7E7B2E08C918F5F1F
:104650008C93009177020A3011F00C941A2380E0B9
:10466000809377025A924A9280E0A42DB52D8C93C4
:1046700081E00E94F7235A924A9282E0A42DB52D40
:104680008C9381E00E94F7230E94B009249682E077
:104690000E94F3235A924A92A42DB52DE0E6FFE43E
:1046A0000E949A248FE00E94F7230E94610A2296BA
:1046B0008FE00E94F3235A924A9280E0A42DB52DF8
:1046C0008C9381E00E94F7235A924A9282E0A42DB3
:1046D000B52D8C9381E00E94F7230E94B0092496A7
:1046E00082E00E94F3235A924A92EFE9F0E0A42D6F
:1046F000B52D0E9447268CE00E94F7230E94610A94
:1047000022968CE00E94F3235A924A9280E0A42DD4
:10471000B52D8C9381E00E94F7235A924A9283E050
:10472000A42DB52D8C9381E00E94F7230E94B0093F
:10473000249682E00E94F3235A924A92A42DB52D2A
:10474000E0E6FFE40E949A248FE00E94F7230E9493
:10475000610A22968FE00E94F3235A924A9280E0E7
:10476000A42DB52D8C9381E00E94F7235A924A9292
:1047700083E0A42DB52D8C9381E00E94F7230E9445
:10478000B009249682E00E94F3235A924A92E8E10B
:10479000F1E0A42DB52D0E94472689E70E94F7235A
:1047A0000E94610A229689E70E94F323EAEEFDE463
:1047B0000E94402482E20E944A24E4EFFDE40E9429
:1047C000402482E20E944A240E94472484E690E02A
:1047D0000E9485240E94C71508958E2E9F2E08954D
:1047E000E82DF92D0895481A8827580A0895480E8B
:1047F0008827581E0895ED91FC91EF5FFF4FFC93C1
:10480000EE9308958F938D918823E9F711978F91F7
:10481000089580919E00882309F081E00895809199
:104820009E00882309F408950F929F93AF93BF933E
:104830007F9380919E008823E1F3F89480919E00FD
:104840008A9580939E0090919C00A0E6B0E0A90F0D
:104850000024B01D8C9193959C3309F49927909373
:104860009C0078947F91BF91AF919F910F90089594
:10487000ACE7B7E08D91882311F00CD0FBCF089501
:104880000E94A024802D11F005D0FACF08958DE06C
:1048900001D08AE05D9BFECF8CB9089588EE93E04D
:1048A00034D03197D9F708953197F1F708950E94E0
:1048B00067248D910E946B249A95D9F70E946A24EF
:1048C0000895DB98D39ADC98D49AD1980895DB9810
:1048D000DC980895089508E0880F10F4DC9A02C06F
:1048E000DC980000DB9A0058005EF0F3DB9800587B
:1048F000005EF0F3C99983950A9571F7089568945D
:1049000062F80895E89462F80895EF93FF93EE2714
:10491000E82BE92B31F0E0EAFFE03197F1F701975E
:10492000D1F7FF91EF9108955A924A92480E882745
:10493000581E08950E94A0240D920020D9F70895D2
:10494000C89531960020089591E0882321F088943D
:10495000991F8A95E9F7892F909508952E2E3F2E5D
:10496000992781918D3209F093958823D1F79A95F3
:10497000E22DF32D112361F0091718F011F0101B2F
:1049800001C0191B28F021F080E28D931A95E9F7F8
:1049900080818D3219F48D93319604C0222311F059
:1049A0008BE28D93091738F031F0091B21F080E379
:1049B0008D930A95E9F781918D938823E1F733234D
:1049C00051F0EA2FFB2F319633958E9182933A95D1
:1049D000E1F78EE28C9308950181082B0183128107
:1049E00019231283EF93FF93E4E0F0E00E94542434
:1049F000FF91EF9108950E947F24FF270E94A42435
:104A0000EBDFEF93FF93ECE7F7E00E945424FF9174
:104A1000EF91182B128309230183EF93FF93E4E6B0
:104A2000F1E00E945424FF91EF911081182369F462
:104A3000EF93FF93ECE7F7E00E945424FF91EF918E
:104A40001081182311F00E948224EF93FF93ECE76A
:104A5000F7E00E945424FF91EF9108950E94A4244E
:104A6000FF2729915D9148E0B7DFEF93FF93E4E0E2
:104A7000F0E00E945424FF91EF91579510F4182B09
:104A80001283EF93FF93ECEEF0E00E945424FF9129
:104A9000EF91182B1283EF93FF93E4E0F0E00E9474
:104AA0005424FF91EF914A95F9F62A95D9F6089585
:104AB0000E94A424FF27299148E055278DDF092370
:104AC0000183EF93FF93E4E1F0E00E945424FF910F
:104AD000EF9188941081182309F008945795EF936B
:104AE000FF93E0EBF0E00E945424FF91EF914A9590
:104AF00029F75D932A9501F708957F930F93AF935C
:104B0000BF938F939F938FB78F9380919E000CE3F9
:104B1000081B21F49CB10E947F2412C000919D00CB
:104B2000A0E6B0E077279CB1A00FB71F9C938395B8
:104B300080939E0003950C3309F4002700939D0099
:104B40008F918FBF9F918F91BF91AF910F917F9167
:104B50001895040F151F261F371F0895000F111FEA
:104B6000221F331F089500951095209530950F5FF3
:104B70001F4F2F4F3F4F0895019110810EC001919B
:104B80001191219130810BC00191108117FF05C057
:104B90003FEF2FEF04C0008111272227332737FF73
:104BA00003C0E1DF8DE28D93CF93DF93CF92DF924D
:104BB000EF92AA24BB24CC24DD24EE2440E2CAE0F8
:104BC000DD2755E093E38881890F87FD9F7083FD82
:104BD000907F891B89935A95A9F7C0DFAA1CBB1C3B
:104BE000CC1CDD1CEE1C4A9551F7E894EFE0FF2742
:104BF00082910ED0EB30E0F71EF068948A2D0CD035
:104C000088278D93EF90DF90CF90DF91CF9108951B
:104C1000982F829501D0892F8F70805D26F0803388
:104C200009F4089568948D93089500271127222789
:104C300033271DD08A3328F4803318F005D015D0DF
:104C4000F9CF0EF490CF089580538F93402F512FBA
:104C5000622F732F83DF82DF7CDF80DF8F919927C4
:104C6000080F191F291F391F08958D910895E89481
:104C7000FCDF8032E9F38B32D9F38930C9F38D320E
:104C800011F46894F2CF089588278D930895819147
:104C90008D938823E1F7089509919191992351F01B
:104CA0008A95D9F7319781918D930A9519F08823C8
:104CB000D1F70895E9CFE199FECFEEBBFFBB319666
:104CC0000895F9DF8D917B3729F48DBBE29AE19A43
:104CD0008823B9F777270895EEDFE09A8DB38D9397
:104CE000882319F09A95C1F79D930895FF93881B27
:104CF000F9E0001FFA9511F4FF910895881F841BB5
:104D000018F4840F8894F5CF0894F3CF8FEF839530
:104D10009D919923E1F70895689401C0E894AF93B9
:104D2000BF938D9116F0919103C00E94A024902D05
:104D3000891718F011F48823A1F7BF91AF91089556
:104D40005265762E3132313033312E6400004753B4
:104D50004D2053494D39303044002D2D2D2D2D2D12
:104D60002D2D2D2D2D2D2D2D000041565270726FA1
:104D70006A6563742E727500C2EAEBFEF7E5EDE832
:104D8000E520202020200000DAFAFAFAFAFAFAFAEE
:104D9000FAFAFAFAFADB0000D900D800D600D700F8
:104DA000D0E5E3E8F1F2F0E0F6E8FF202020000093
:104DB000DA00CEF7E8F1F2EAE020E1F3F4E5F0E022
:104DC000000041540000C2E5F0E8F4E8EAE0F6E84B
:104DD000FF20415400004F4B0000D3E4E0EBE5ED31
:104DE000E8E520534D532020000041542B434D470C
:104DF00044413D0044454C20414C4C00C9005349BE
:104E00004D3930304420E3EEF2EEE221000041540F
:104E10002B434D47463D310041542B434C49503DB7
:104E200031003000310032003300340035003600EC
:104E3000370038003900410042004300440045007B
:104E400046004700480049004A004B004C004D0016
:104E50004E004F00500051005200530054005500C6
:104E600056005700580059005A0061006200630064
:104E70006400650066006700680069006A006B00F6
:104E80006C006D006E006F007000710072007300A6
:104E90007400750076007700780079007A00C00011
:104EA000E000C100E100C200E200C300E300C40072
:104EB000E400C500E500A800B800C600E600C70091
:104EC000E700C800E800E900CA00EA00CB00EB00F8
:104ED000CC00EC00CD00ED00CE00EE00CF00EF00E6
:104EE000D000F000D100F100D200F200D300F300B6
:104EF000D500F500F700F600D400F400F800F90042
:104F0000DC00FC00FA00DB00FB00DD00FD00DE0041
:104F1000FE00DF00FF0020002D002E003A003E00C2
:104F2000B0004000260027003C002A002C0024008E
:104F30003D002100BD00230028005B0025002B0060
:104F40005E003F005D0029003B002F005C005F0019
:104F50002B434D54000041542B434D47523D00001C
:104F60002020202020202020202020202020000081
:104F70004F6666004C6F6164204F4646202020201B
:104F8000202000004F4E00004C6F6164204F4E20E7
:104F90002020202020200000415453303D300000CC
:104FA000415453303D32000046697273746E756D22
:104FB000626572004E756D6265723A200000204F86
:104FC0004B0053494D393030440054656D703A0000
:104FD0004C6F61643A005049522073656E736F7272
:104FE0003A0053656E6420534D532066726F6D20F6
:104FF00073656E736F72733A000041542B434D47D3
:10500000533D00006572726F7200B043000041545E
:105010002B434F50533F00002020202020202020F1
:105020002020200041542B43535100002020000039
:105030003E2000003C2000003C4000003C260000D8
:1050400041542B43434C4B3F000041544400C7E2C2
:10505000EEEDE8EC20EDE000C7E0EFF0EEF120E14E
:10506000E0EBE0EDF1E000004154442A3130302320
:10507000000053494D39303044204F4E202020202D
:10508000000053494D39303044204F464600C4E0BB
:10509000F22E203120200000416C61726D21000051
:1050A000CEF2EFF0E0E2EAE020534D532020000082
:1050B000C4E0F22E203020200000596573004E6FAE
:1050C000000041542B434D47523D31002B434D4787
:0250D0000000DE
:00000001FF
